:100000000EC028C04DC026C025C025C023C022C0B8
:1000100021C020C01FC01EC01DC01CC01BC0112499
:100020001FBECFE5D1E0DEBFCDBF10E0A0E6B0E05F
:10003000E6EAF4E003C0C89531960D92AA36B107FE
:10004000D1F710E0AAE6B0E001C01D92A03BB107D5
:10005000E1F7A2C0D5CF1F920F920FB60F921124D5
:100060008F939F93AF93BF938091AC009091AD001D
:10007000A091AE00B091AF000196A11DB11D80937B
:10008000AC009093AD00A093AE00B093AF00BF91D1
:10009000AF919F918F910F900FBE0F901F90189569
:1000A0001F920F920FB60F9211242F933F934F93ED
:1000B0005F938F939F93AF93BF93CF93DF93EF9310
:1000C000FF93B49B47C022B78091AC009091AD00E4
:1000D000A091AE00B091AF0008B601FE04C022B7F7
:1000E0000196A11DB11DDA2FC92FB82FAA27A20F83
:1000F000B11DC11DD11DC19A80916B0090916A0004
:10010000891B803198F080916A00E82FFF27EF70FB
:10011000F070EE0FFF1FEE0FFF1FE659FF4F228119
:100120003381448155818F5F80936A0080916B0099
:10013000E82FFF27EF70F070EE0FFF1FEE0FFF1F8D
:10014000E659FF4FA283B383C483D5838F5F809327
:100150006B0001C0C198FF91EF91DF91CF91BF91EA
:10016000AF919F918F915F914F913F912F910F9000
:100170000FBE0F901F901895382F21E097E0C2987E
:10018000832F822311F4C09801C0C09AC29A220F13
:10019000915097FFF4CF0895CFE5D1E0DEBFCDBFFA
:1001A000EE24FF24002711272E2C3F2C402E512E09
:1001B0008E2C9F2CA02EB12EDD24CD2CB89ABA9A6D
:1001C000BB9AB99ABC98C49ADABC82E083BF8BB759
:1001D00080628BBFAC9A89B7826089BFE092AC0025
:1001E000F092AD000093AE001093AF00789484EFCE
:1001F00091E0AAEFB0E01197F1F70197D1F788B33A
:1002000098E0892788BBF89460916B0080916A0020
:10021000681B623008F44CC080916B00E82FFF2708
:100220003197EF70F070EE0FFF1FEE0FFF1FE659D2
:10023000FF4FE280F3800481158180916B00E82FED
:10024000FF273297EF70F070EE0FFF1FEE0FFF1FCA
:10025000E659FF4F82809380A480B580B2E0DB2E08
:10026000512F402F3F2D2E2D2854384E41405040C5
:10027000D616F0F480916B00E82FFF27ED19F109F5
:100280003197EF70F070EE0FFF1FEE0FFF1FE65972
:10029000FF4F82819381A481B58182179307A407C0
:1002A000B50730F0882E992EAA2EBB2ED394E0CF1E
:1002B000789421E02D1508F095C0E214F3040405AC
:1002C000150531F4C20E84E08C1508F090CF8AC079
:1002D000CC242E2C3F2C402E512E8D2D992701976A
:1002E000AA2797FDA095BA2F20EE30E742E750E00D
:1002F000682F792F8A2F9B2F7ED0B92FA82F972F69
:10030000862F512F402F3F2D2E2D281939094A09AC
:100310005B09682F792F8A2F9B2F9ED0B52FA42F92
:10032000932F822FAA27BB27D92FC82F41E0742EE5
:1003300027E28031920740F064E670E077D0D72F53
:10034000C62F80E819DF7C2C8C2F9D2F6AE070E08F
:100350006DD0F92FE82FE05AFF4F80810DDFCA30B2
:10036000D10580F08C2F9D2F6AE070E05FD0972F31
:10037000862F6AE070E05AD0F92FE82FE05AFF4F3D
:10038000808101C08C2DF8DEC436D10580F08C2F21
:100390009D2F64E670E04AD0972F862F6AE070E0C8
:1003A00045D0F92FE82FE05AFF4F808101C080E04F
:1003B000E3DE772009F41BCF83E0C83ED80780F046
:1003C0008C2F9D2F68EE73E031D0972F862F6AE037
:1003D00070E02CD0F92FE82FE05AFF4F808109C040
:1003E00080E007C080E8C8DE80E8C6DE80E8C4DEC2
:1003F00080E8C2DEFCCEFF27EE27BB27AA2760FFDE
:1004000004C0A20FB31FE41FF51F220F331F441FA8
:10041000551F969587957795679589F70097760785
:1004200071F79F2F8E2F7B2F6A2F0895AA1BBB1B5E
:1004300051E107C0AA1FBB1FA617B70710F0A61BE4
:10044000B70B881F991F5A95A9F780959095682F2B
:10045000792F8A2F9B2F0895A1E21A2EAA1BBB1B6E
:10046000EA2FFB2F0DC0AA1FBB1FEE1FFF1FA217F5
:10047000B307E407F50720F0A21BB30BE40BF50B61
:10048000661F771F881F991F1A9469F760957095EA
:1004900080959095262F372F482F592F6A2F7B2F25
:0604A0008E2F9F2F08952E
:0A04A6007E18B6BCD8ECEE38FEFC60
:00000001FF
